:020000000DC031
:0200020018954F
:02000C007EC0B4
:0200140018953D
:10001C00F8940FED0DBF0FEF01BB08E707BB00E035
:10002C0008BB0FE702BBC39AC49AC59A00E008B993
:10003C0001E003BF02E009BF442755276627772755
:10004C0088279927AA27F894BA9A0EE10A95F1F70E
:10005C00002702BF0FEF08BFBA9878944599FECFDE
:10006C00F89412B70FE702BBC39AC49AC59A00273B
:10007C00FF27E12FE40FF01FE50FF01FE60FF01F35
:10008C00E70FF01FE80FF01FE90FF01FEA0FF01F4A
:10009C00F695E795F695E795F695E795452F562F46
:1000AC00672F782F892F9A2FA12FE231A0F0EC31F6
:1000BC00A0F0E932A0F0E633A0F0E434A0F0E13592
:1000CC00A0F0EF35A0F0EE36A0F0EC37A0F0EB3856
:1000DC00A0F0C598B8CF9098B6CF9198B4CF92981D
:1000EC00B2CF9398B0CF9498AECF9598ACCF96985A
:1000FC00AACFC398A8CFC498A6CFC598A4CF0FE712
:10010C0002BBC39AC49AC59AC5980FED0DBF9BCF7D
:00000001FF
